S018000064656D6F70726F675F786D63343730302E737265633D
S3150800C0008890FE1F79FF0008C1FF0008C5FF0008D9
S3150800C010C9FF0008CDFF0008D1FF00080000000096
S3150800C020000000000000000000000000D5FF000826
S3150800C030D9FF000800000000DDFF000887E40008BB
S3150800C040E1FF0008E5FF0008E9FF0008EDFF00082A
S3150800C050F1FF0008F5FF0008F9FF0008FDFF0008DA
S3150800C06001000108000000000000000000000000B8
S3150800C0700500010800000000090001080D0001087C
S3150800C0801100010815000108190001081D00010822
S3150800C0902100010825000108290001082D000108D2
S3150800C0A03100010835000108390001083D00010882
S3150800C0B04100010845000108490001084D00010832
S3150800C0C05100010855000108590001085D000108E2
S3150800C0D06100010865000108690001086D00010892
S3150800C0E07100010875000108790001087D00010842
S3150800C0F08100010885000108890001088D000108F2
S3150800C1009100010895000108990001089D000108A1
S3150800C110A1000108A5000108A9000108AD00010851
S3150800C120B1000108B5000108B9000108BD00010801
S3150800C130C1000108C5000108C9000108CD000108B1
S3150800C140D1000108D5000108D9000108DD00010861
S3150800C150E1000108E5000108E9000108ED00010811
S3150800C16000000000000000000000000000000000C1
S3150800C170F1000108F5000108F9000108FD000108B1
S3150800C1800101010805010108090101080D0101085D
S3150800C1901101010815010108190101081D0101080D
S3150800C1A02101010825010108290101082D010108BD
S3150800C1B03101010835010108390101083D0101086D
S3150800C1C04101010845010108490101084D0101081D
S3150800C1D05101010855010108590101080000000034
S3150800C1E05D0101086101010865010108690101088D
S3150800C1F06D0101080000000071010108000000003F
S3150800C200EE11AA55C2788A18DFF83833DA708378BF
S3150800C2100A0092B2120AD218DFF828339A704278C6
S3150800C220DFF820335A700078DFF818231070DFF82B
S3150800C23014038278080080B2000A80B2824212DAB9
S3150800C240DFF800034078401CDFF8F8225070DFF86A
S3150800C250F4024078002806D1DFF8E8020078401C8E
S3150800C260DFF8E0221070DFF8DC02C07889B201F04E
S3150800C270FF0188421EDADFF8CC028078401CDFF81E
S3150800C280C4128870DFF8BC028078002812D1DFF863
S3150800C290B4024078401CDFF8AC124870DFF8A402FC
S3150800C2A04078002806D1DFF89C020078401CDFF8A9
S3150800C2B094120870704710B492B20A44531E0BE0E9
S3150800C2C00A7812024C78121910180400A4B292B215
S3150800C2D0944200D2401C891C9942F1D3994208D154
S3150800C2E009780A021018010089B292B2914200D266
S3150800C2F0401C80B210BC704780B51422DFF8481283
S3150800C3000020FFF7D8FF80B2002802D14FF6FF7051
S3150800C31002E080B201F036FA80B202BD10B5DFF84D
S3150800C3202C12097C0902DFF82422527C8918B1F103
S3150800C330140454FA80F00822DFF8141280B2FFF7CA
S3150800C340BAFF220092B2DFF80C1280B2FFF7B3FFF1
S3150800C35080B2002802D14FF6FF7002E080B201F0E9
S3150800C36011FA80B210BD80B50620FFF7D7FF02BDCF
S3150800C3700020DFF8E41108700EE00020DFF8DC1179
S3150800C380DFF8D421127821F81200DFF8CC01007802
S3150800C390401CDFF8C4110870DFF8BC0100780028DB
S3150800C3A0EBD000206C4908700CE000206C496A4A02
S3150800C3B012781E235A431144487667480078401C71
S3150800C3C065490870644800780028EED04FF480600C
S3150800C3D0644908800020604908700CE00020624922
S3150800C3E05D4A127840235A43114488805A48007897
S3150800C3F0401C59490870584800780028EED0704704
S3150800C40070B504000D000CE05748534909784022DE
S3150800C4105143084486885348008801F0B3F9864298
S3150800C42011D150480088401C4E4908804D48008864
S3150800C430B0F5FA4F03DB4FF480504A4908800020D4
S3150800C4404549087004E044480078401C4249087091
S3150800C450414800780028D7D0002600203E490870B9
S3150800C46004E03D480078401C3B4908703A4800788B
S3150800C47000280FD13C4838490978402251430844DE
S3150800C48080880028EDD1384833490978402251433D
S3150800C49000EB0106002E01D1002018E03148008883
S3150800C4A03049098889B2090A51EA0020B080F58026
S3150800C4B0002C05D104210022300001F097F903E091
S3150800C4C0208830806088708040203072300070BDCF
S3150800C4D00021214A117004E01F490978491C1E4AA7
S3150800C4E011701D49097800290CD11C491A4A12787D
S3150800C4F031F812100029EFD11849174A127821F895
S3150800C5001200FFE7704780B5010089B21748006836
S3150800C5100830FFF777FE0B48007814490968087257
S3150800C52008484078114909684872064880780F49D2
S3150800C530096888720348C0780C490968C87201BD41
S3150800C540000000005088FE1F7E80FE1F7080FE1FC0
S3150800C5508A80FE1F9280FE1F6888FE1F5C88FE1F69
S3150800C560F087FE1F6088FE1F5887FE1F4488FE1F3F
S3150800C57010B5DFF8141E0C68C0B2042806D1DFF81F
S3150800C5803C0E0088002840F061821DE0DFF8301E6E
S3150800C590DFF8302E1160DFF82C1E0968DFF8282E28
S3150800C5A01160C0B2032818D1607E10F00F0003286E
S3150800C5B00AD1208A002807D10820DFF8281E08702B
S3150800C5C001F094F900F0A9BF0020DFF81C1E0880CE
S3150800C5D00020DFF8101E087010BDC0B2022840F017
S3150800C5E0D180DFF8080EC078401CDFF8001EC8703E
S3150800C5F0DFF8F80DC07800281ED1DFF8F00D807836
S3150800C600401CDFF8E81D8870DFF8E00D8078002808
S3150800C61012D1DFF8D80D4078401CDFF8D01D4870DD
S3150800C620DFF8C80D4078002806D1DFF8C00D00787D
S3150800C630401CDFF8B81D08700020DFF8AC1D088024
S3150800C6400020DFF8781D0880607E072802D0607E0B
S3150800C650052808D1A07E401CA076A07E782801D1A6
S3150800C66000206076B0E7607E0028FBD0208A00288C
S3150800C6707AD0A07E411EA176C0B20028F2D1E07E13
S3150800C680082808D0607E022802D0607E012810D1D2
S3150800C690E07E05280DD1002060768020DFF8441D55
S3150800C6A0087001F023F91420DFF8B01D81F82F0077
S3150800C6B0B0E2E07E052801DB042000E0E07E0321ED
S3150800C6C011FA00F0A076E07E401CE076607E10F05D
S3150800C6D00F00C0B201280AD0022835D0032839D065
S3150800C6E004283FD006283DD008283BD0BAE71020BA
S3150800C6F0DFF8681D81F82F00DFF8600D90F82F002D
S3150800C70050F00200DFF8541D81F82F000220DFF8F0
S3150800C7104C1D81F836000420DFF8401D81F83700EB
S3150800C7200620DFF8381D81F838000A20DFF82C1DAE
S3150800C73081F839002C20DFF8B01C08806020DFF86B
S3150800C7401C1D81F82E006EE20020DFF8101D81F80E
S3150800C7502F00D1E70420DFF88C1C087001F0C6F81A
S3150800C76000F01FBF00F074BE607E10F00F000328B3
S3150800C7707FF478AF0820DFF86C1C087001F0B6F873
S3150800C78000F0CBBEC0B2052826D1DFF8040E00683B
S3150800C790808800281FD00020DFF8EC1B0860DFF82F
S3150800C7A0F40DDFF8201C0860DFF8180C0068DFF8C5
S3150800C7B0181C08600020DFF8041C0880DFF8FC0B52
S3150800C7C00088DFF8241C08800820DFF8181C087089
S3150800C7D001F0EBFBD3E6F7E6DFF8800C807B452813
S3150800C7E07FF4F2AEDFF8000C0088DFF8701C097CD5
S3150800C7F00902DFF8682C527C8918884216DBDFF8B4
S3150800C8005C0C007C0002DFF8541C497C4018DFF8F9
S3150800C810D81B0880DFF8440C007D3F21084204D16C
S3150800C820DFF8380C407D002801D0CDE6CCE6DFF8ED
S3150800C830B80D0088DFF8B41D0988884207D1DFF8EB
S3150800C840A80D4088DFF8A41D4988884210D0DFF873
S3150800C8500C0CC08BDFF8901D0988884207D1DFF8D9
S3150800C860FC0B008CDFF8801D4988884200D0ABE6B7
S3150800C870FFF742FD4FF6FF7188427FF4A5AEDFF859
S3150800C880DC0BC07D062809D1FFF76DFD4FF6FF7159
S3150800C890884240F03D81DFF8584D3BE1DFF8BC0B9C
S3150800C8A0C07D11280CD1DFF8400B00881C38DFF852
S3150800C8B0381B0880DFF8080EDFF8D41C086048E04B
S3150800C8C0DFF8980BC07D01287FF47EAEDFF88C0B6D
S3150800C8D090F8220008287FF477AE0020DFF87C1B4A
S3150800C8E081F82200DFF8740B808C4FF6F7718842C6
S3150800C8F007DBDFF8680B808C0930DFF8601B88845B
S3150800C90006E0DFF8580B808C0830DFF8501B888467
S3150800C910DFF8480B408BDFF8441BC883DFF83C0B75
S3150800C920808BDFF8381B0884DFF8BC0C0088DFF83A
S3150800C9302C1B4883DFF8B00C4088DFF8201B88835F
S3150800C94000F019BFDFF8480C00684030DFF8401CDB
S3150800C9500860DFF83C0C0068DFF8681D884274D26E
S3150800C960DFF82C0C006880880028EBD0DFF8EC0A8A
S3150800C970808CDFF81C1C096889888842E2D1DFF8B8
S3150800C980100C0068C08800280FD0DFF8D00A408C49
S3150800C990DFF8FC1B0968C988884206D0DFF8F00B67
S3150800C9A00068C088B0F58A4FCCD1DFF8E40B006880
S3150800C9B00088DFF8381C0988884208D1DFF8D00BD0
S3150800C9C000684088DFF8241C4988884223D0DFF8AD
S3150800C9D0C00B00680088DFF8A81D0988884208D1BE
S3150800C9E0DFF8AC0B00684088DFF8941D4988884258
S3150800C9F011D0DFF8680A408BDFF8941B09680988AC
S3150800CA0088429FD1DFF8540A808BDFF8841B0968B7
S3150800CA104988884296D10020DFF86C190860022000
S3150800CA20DFF8C0190870DFF86C0BDFF89819086092
S3150800CA30DFF890090068DFF8901908600020DFF831
S3150800CA407C19088001F0B1FA99E5BDE5DFF86C09B3
S3150800CA5000881C30DFF890190880DFF88C090088F8
S3150800CA6080B2000ADFF8F4190874DFF87C09008838
S3150800CA70DFF8E8194874DFF8180B0068007ADFF861
S3150800CA80DC1988751120DFF8D419C875DFF82C0968
S3150800CA9000880830DFF824190988083189B2090A9C
S3150800CAA051EA0020DFF8B419C8840020DFF8AC1971
S3150800CAB00885DFF8DC0A00688088DFF8A019488452
S3150800CAC0DFF8CC0A0068C088DFF890198884DFF898
S3150800CAD0180B0088DFF884194883DFF80C0B4088A8
S3150800CAE0DFF878198883DFF8A80A00680088DFF875
S3150800CAF06C19C883DFF8980A00684088DFF85C1963
S3150800CB000884DFF8BC08DFF8BC18086000F00FBE20
S3150800CB105AE51E34DFF8D80AA042C0F0DF80607EEE
S3150800CB200028F6D0DFF83409808CA1888842F0D135
S3150800CB30DFF82809408CE1888842EAD1DFF81C0929
S3150800CB40408B21888842E4D1DFF81009808B618800
S3150800CB508842DED1DFF8300804600020DFF8841848
S3150800CB600870DFF8F80890F82F00400700F1CD822A
S3150800CB70DFF8E80890F82E00C0B200098000DFF858
S3150800CB80381C0870DFF860080088DFF82C1C097864
S3150800CB90401A1438DFF850180880607E10F00F002D
S3150800CBA0022808D1DFF8B40890F82F0010F03F00EB
S3150800CBB0122800F0B382DFF830080088002807D171
S3150800CBC0DFF8980890F82F000321084200F0A682A3
S3150800CBD0DFF8880890F82600217A884215D1DFF810
S3150800CBE07C0890F82700617A88420ED1DFF86C0835
S3150800CBF090F82800A17A884207D1DFF8600890F8F3
S3150800CC002900E17A884200F089821020DFF84C1862
S3150800CC1081F82F002820DFF8D01708805020DFF889
S3150800CC203C1881F82E00207ADFF8301881F82A009F
S3150800CC30607ADFF8281881F82B00A07ADFF81C182C
S3150800CC4081F82C00E07ADFF8141881F82D00207B93
S3150800CC50DFF8081881F82600607BDFF8001881F8ED
S3150800CC602700A07BDFF8F41781F82800E07BDFF8BF
S3150800CC70EC1781F829000620DFF8E017C875A088A8
S3150800CC80DFF8D8174884E088DFF8D0178884DFF8FB
S3150800CC9058090088DFF8C4174883DFF84C0940882C
S3150800CCA0DFF8B81788832088DFF8B017C88360884C
S3150800CCB0DFF8A8170884607EC00640F111850020B9
S3150800CCC0DFF8981781F83100DFF8900790F83100FF
S3150800CCD0DFF8881781F8300000F00ABDDFF87C0716
S3150800CCE090F82F0010F03F00022806D0DFF86C07F6
S3150800CCF090F82F00400729D566E4DFF86007808C96
S3150800CD00DFF8B81A08800020DFF8AC1A087006E0C9
S3150800CD10DFF8A40A0078401CDFF89C1A0870DFF8D0
S3150800CD20980A00780028E1D1DFF8900A0088DFF831
S3150800CD30901ADFF8842A127831F812108842E7D15F
S3150800CD4000240020DFF8701A0870F0E01420DFF8DD
S3150800CD500C1781F82F002820DFF88C160880502041
S3150800CD60DFF8F81681F82E00DFF8F00690F82900AB
S3150800CD70DFF8441A0870DFF8E40690F82D00DFF8AB
S3150800CD80DC1681F82900DFF8300A0078DFF8CC16BF
S3150800CD9081F82D00DFF8C40690F82800DFF8181A85
S3150800CDA00870DFF8B80690F82C00DFF8B01681F89E
S3150800CDB02800DFF8040A0078DFF8A01681F82C00AE
S3150800CDC0DFF8980690F82700DFF8EC190870DFF806
S3150800CDD08C0690F82B00DFF8841681F82700DFF818
S3150800CDE0D8090078DFF8741681F82B00DFF86C068E
S3150800CDF090F82600DFF8C0190870DFF8600690F88A
S3150800CE002A00DFF8581681F82600DFF8AC09007802
S3150800CE10DFF8481681F82A00DFF8400690F82D005A
S3150800CE20401CDFF8381681F82D00DFF8300690F838
S3150800CE302D00002826D1DFF8240690F82C00401C87
S3150800CE40DFF8181681F82C00DFF8100690F82C0089
S3150800CE50002817D1DFF8040690F82B00401CDFF8ED
S3150800CE60FC1581F82B00DFF8F40590F82B00002854
S3150800CE7008D1DFF8E80590F82A00401CDFF8DC1531
S3150800CE8081F82A00DFF8D405408CDFF830190880CD
S3150800CE90DFF8C805808CDFF8C4154884DFF81C095C
S3150800CEA00088DFF8B8158884DFF8B005408BDFF80E
S3150800CEB0AC15C883DFF8A405808BDFF8A0150884B5
S3150800CEC0DFF824070088DFF894154883DFF8180789
S3150800CED04088DFF88815888300F00ABCDFF8100759
S3150800CEE0DFF8D41809781E2251430844407E0728E3
S3150800CEF016D1002C0BD0A07EDFF8F416DFF8B82880
S3150800CF0012781E235A431144897E884208D2DFF8D4
S3150800CF10E006DFF8A41809781E22514300EB010445
S3150800CF20DFF894080078401CDFF88C180870DFF8E2
S3150800CF3088080078002813D1DFF8B406DFF87818D7
S3150800CF4009781E2251430844407E0028C6D1DFF8DE
S3150800CF50A006DFF8641809781E22514300EB010485
S3150800CF60002C3FF431ABDFF8200404600320A076E0
S3150800CF70A07E20760020A0750420E0750020E076CB
S3150800CF80DFF8D804808CA080DFF8D004408CE080DD
S3150800CF90DFF8C804408B2080DFF8C004808B6080EF
S3150800CFA001206076DFF8440400782073DFF83C043B
S3150800CFB040786073DFF834048078A073DFF82C04B7
S3150800CFC0C078E07301202082DFF8900490F82900E9
S3150800CFD0E072DFF8880490F82800A072DFF87C0475
S3150800CFE090F827006072DFF8740490F82600207223
S3150800CFF00120FFF788FADFF8640490F82E0010F095
S3150800D000F0005128FFF673AB0020DFF8AC17087064
S3150800D01006E0DFF8A4070078401CDFF89C170870C4
S3150800D020DFF894070078DFF8341491F82E10C9B2A7
S3150800D0300909C9B2491FB0EB810FBFF658ABDFF833
S3150800D0401C04DFF874170978084490F83600DFF8EE
S3150800D05074170870DFF86C07007800283FF447ABB0
S3150800D060DFF8600700780128D3D0DFF85807007882
S3150800D07002282FD1DFF8E403DFF83C1709780844C3
S3150800D08090F83700042825D1DFF8D003DFF82817F1
S3150800D0900978084490F83800DFF8C013DFF8182735
S3150800D0A01278114491F8391051EA0020DFF80C176C
S3150800D0B00880DFF80807008840F20B61884202DB27
S3150800D0C040F20A6002E0DFF8F40600886082A08277
S3150800D0D0FFF70DBBDFF88403DFF8DC160978084490
S3150800D0E090F8370000283FF402ABDFF8CC0600784A
S3150800D0F0DFF86813DFF8C0261278114491F8371064
S3150800D1000818DFF8B41608708AE700206076202031
S3150800D110B449087000F0EAFBFFF756BACF4890F812
S3150800D1202F00C0065FD5208A00285CD0218A14F11A
S3150800D1300C00FFF767F8C94890F82A00DFF8881648
S3150800D140097888424FD1C54890F82B00DFF8781641
S3150800D1504978884247D1C14890F82C00DFF868160C
S3150800D160897888423FD1BD4890F82D00DFF85816D7
S3150800D170C978884237D1DFF8500600782073DFF87F
S3150800D180480640786073DFF840068078A073DFF8B9
S3150800D1903806C078E073E07E00281DD194F918009F
S3150800D1A094F91A10401AA17DC9B2B0EBD100A17D3D
S3150800D1B04118A17540B2002801D540B24042E17D30
S3150800D1C0C9B2B0EB9100E17D4018E075A07DC0B210
S3150800D1D0E17D11EBD0002076012082490870207E7F
S3150800D1E0A07600202082607E10F00F00C0B20128D1
S3150800D1F013D0C0F07382032800F0FA802ED30528D6
S3150800D20000F03B82C0F00482072800F05D82C0F07F
S3150800D2105D82082800F0F08160E272480078C00755
S3150800D2201AD50320607640206E49087000202082B7
S3150800D2306D480088002809D06A48007850F0020036
S3150800D2406849087068480088FFF75DF900205B495F
S3150800D250088000F04BFB60E1FFF7B6B9614800783B
S3150800D260C00740F1B3807D4890F82F0010F03F00CA
S3150800D270122840F0AB80794890F82E0010F0F000A4
S3150800D280512827DB0020DFF83015087006E0DFF8A4
S3150800D29028050078401CDFF820150870DFF8180507
S3150800D2A000786E4991F82E10C9B20909C9B2491F0A
S3150800D2B0B0EB810F0EDA6948DFF8FC1409780844E8
S3150800D2C090F83600DFF8FC140870DFF8F8040078E8
S3150800D2D0002822D103206076604890F82600207244
S3150800D2E05E4890F8270060725C4890F82800A072A3
S3150800D2F05A4890F82900E0720120FFF704F9422005
S3150800D300384908700020208200203749088000200C
S3150800D3102A49088000F0EAFAFFE0DFF8A804007856
S3150800D3200128B4D0DFF89C04007802282ED14B4897
S3150800D330DFF884140978084490F83700042825D1C2
S3150800D3404648DFF874140978084490F838004349C9
S3150800D350DFF864241278114491F8391051EA002054
S3150800D360DFF858140880DFF85404008840F20B618F
S3150800D370884202DB40F20A6002E0DFF840040088D7
S3150800D3806082A082A6E700BF4488FE1F3348DFF804
S3150800D39028140978084490F8370000289AD0DFF84E
S3150800D3A0180400782D49DFF810241278114491F8F2
S3150800D3B037100818DFF8001408706FE75A88FE1F40
S3150800D3C0A680FE1F3C88FE1F4088FE1F20200549B8
S3150800D3D0087000F08BFA0020DFF8F0130968487629
S3150800D3E084E400BF6788FE1F5888FE1F4C88FE1F0E
S3150800D3F01A4890F82F00C00732D5607EC0062FD491
S3150800D400208A00287FF4E0A8DFF8C4030088401CBF
S3150800D41080B2FFF778F8DFF8BC03007850F0100008
S3150800D420DFF8B0130870DFF8A8030088002807D0D3
S3150800D430DFF8A003007850F00200DFF898130870B0
S3150800D44000F054FA01202082082060760020E07659
S3150800D4501120024981F82F00FFF7DCBB7080FE1F00
S3150800D460DFF8740390F82F00800621D5DFF86C03E7
S3150800D4700068DFF8641391F83410DFF85C2392F83B
S3150800D480352052EA01210844DFF850130860DFF816
S3150800D49040030088DFF8401391F83410DFF838238A
S3150800D4A092F8352052EA0121401ADFF82413088041
S3150800D4B0DFF81C03008800280CD0607EC00609D45B
S3150800D4C0C448007850F00200C2490870C048008875
S3150800D4D0FFF719F8C04890F830000002BE4991F8E5
S3150800D4E031104018B5490880A08AB449098888428D
S3150800D4F003D3B2480088002802D1A08AAF49088021
S3150800D500AE4800886082B34800780321084271D08B
S3150800D5100020B349088000F0E9F9AE480078800693
S3150800D5200AD50020AE490880002060761420AA4952
S3150800D53081F82F00FFF76EBBA6480078C0060ED507
S3150800D5400020A74908800120208204206076002058
S3150800D550E0761120A04981F82F00FFF75BBBA048B1
S3150800D560008800281BD09B480078C00701D50020FA
S3150800D5702082208A00280FD1608A99490988884222
S3150800D58002D2608A9649088095480088208206E07B
S3150800D5904888FE1F9A80FE1F208A9149088000202D
S3150800D5A0E076904800688D4908608D480088002814
S3150800D5B00CD0208A002809D0208A2830844908807F
S3150800D5C01820854981F82F00FFF728BB8148007885
S3150800D5D080070FD528207E49088010207E4981F8CB
S3150800D5E02F00FFF71BBB00BF3088FE1FB8FF0008DF
S3150800D5F0F087FE1FFEF7E8BF76480078C00706D515
S3150800D6000020607610207349087000F06FF965E015
S3150800D6106F480088002803D06D480088FEF773FF1E
S3150800D6206D4890F82F00C00716D56A480078C007DD
S3150800D63006D5072060760020A0760020208201E02B
S3150800D640062060760120FEF75EFF1020614908700B
S3150800D65000F04CF9FFF7D9BA5E480078C00705D53F
S3150800D6600520607600202082FEF7AEBF5848008865
S3150800D67000287FF4CAAAFEF7A7BF554800880028E5
S3150800D68003D053480088FEF73EFF534890F82F0012
S3150800D690C0070DD5072060760020A0760120FEF78A
S3150800D6A032FF10204B49087000F020F9FFF7ADBA99
S3150800D6B04748008800287FF4A8AAFEF785BF00BF60
S3150800D6C05887FE1F9887FE1FFFF79FBA41480078C4
S3150800D6D0C00703D5072060760020A076FEF774BF42
S3150800D6E006203D4981F830000A203B4981F831007F
S3150800D6F04020394988753648008880B2000A36497C
S3150800D700087433480088344948740020324981F83F
S3150800D7103500314890F835002F4981F8340000204B
S3150800D7202D494886FEF71FFEC0432B4948864520EB
S3150800D7302949887300202849C87300202649487556
S3150800D7402548407D2449087527480088401C2649F5
S3150800D75008802548008880B2000A1F498874224834
S3150800D76000881D49C87400201B490883FEF7C4FDBC
S3150800D770C04319490883002016490870FEF72CBFD4
S3150800D780B4FF0008010089B2090A51EA002080B2F4
S3150800D790704710B501290DDB114A11801149096836
S3150800D7A0884207D00E490A880E490C6801002000F5
S3150800D7B000F046FC10BD00006888FE1F6288FE1F48
S3150800D7C05C88FE1F6988FE1F5088FE1F4488FE1F5E
S3150800D7D05888FE1F6788FE1F7080FE1F3C88FE1F44
S3150800D7E05A88FE1F4088FE1F5E88FE1F62F30F22BE
S3150800D7F062F31F42401810F0030308D0C91A1FD35A
S3150800D800DB0748BF00F8012D28BF20F8022D1300BA
S3150800D81030B414461546103928BF20E93C00FAD81A
S3150800D820490728BF20E90C0048BF40F8042D8900A5
S3150800D83028BF20F8022D48BF00F8012D30BC7047DC
S3150800D840C91818BF00F8012DCB0728BF00F8012D0D
S3150800D8507047000080B500F087FC00F011FE10F557
S3150800D860FA707049086000F00BFE00F51C50103085
S3150800D8706D490860FEF77CFD0020ADF80000002029
S3150800D880ADF80200BDF8000068490880BDF802003E
S3150800D890664948800020ADF800000020ADF8020077
S3150800D8A0BDF8000062490880BDF80200604948805A
S3150800D8B00020ADF800000020ADF80200BDF8000019
S3150800D8C05C490880BDF802005A4948804EF60300B4
S3150800D8D0FEF7FEFD00F0C2FC574800F012FD0621D7
S3150800D8E0554800F03EFB00F064FB01BD80B5534887
S3150800D8F00078400612D45148007880070ED5504863
S3150800D9000068001D0178FF2908D14078002805D154
S3150800D9100121002000F0E0FD00F09FFE01BD10B5DA
S3150800D92000F0FCFC00282DD0464908804FF4006022
S3150800D930FFF728FF4449898980B281420ED1012028
S3150800D940FEF716FE3F48008800281BD001F048F96C
S3150800D95000F0F8FC00203B49088013E040F606007A
S3150800D960FFF710FF3849898980B281420AD101F050
S3150800D970CDF834480088002804D000F0E3FC0020E5
S3150800D9803049088000F07CFD26490968884239D369
S3150800D9902448006810F5FA7022490860002415E04A
S3150800D9A02A481E2101FB04F108442949086002207F
S3150800D9B0FEF7DEFD23480088002806D001F010F99E
S3150800D9C000F0C0FC00201F490880641C002CE7D02A
S3150800D9D0002415E01F48402101FB04F108441E49B4
S3150800D9E008600520FEF7C4FD16480088002806D002
S3150800D9F001F0F6F800F0A6FC002012490880641C25
S3150800DA00002CE7D000F03CFD07490968884208D396
S3150800DA100548006800F51C5010300349086000F0FE
S3150800DA209DFF10BD2488FE1F2888FE1F3088FE1F14
S3150800DA303888FE1F3488FE1F1088FE1F6788FE1F61
S3150800DA403C88FE1F5888FE1F7080FE1FF087FE1F49
S3150800DA504488FE1F5887FE1F4888FE1F352202701D
S3150800DA60401C01220270401C0170401C704710B512
S3150800DA70040036202070641C04202070641C0422D4
S3150800DA80DFF87815200000F0DBFA201D10BD10B570
S3150800DA90040032202070641C04202070641C0422B8
S3150800DAA0DFF85C15200000F0CBFA201D10BD3721E9
S3150800DAB00170401C03210170401C01210170401CAB
S3150800DAC003210170401C06210170401C7047FF218C
S3150800DAD00170401C704738B50400012020700120F1
S3150800DAE06070DFF820058069A0700020E0700422CD
S3150800DAF0DFF81415251D280000F0A2FA0020208161
S3150800DB00802060810422DFF8041514F10C05280032
S3150800DB1000F096FA0421002214F110052800FFF7F8
S3150800DB2065FE0421002214F114052800FFF75EFEA5
S3150800DB300421002214F118052800FFF757FEDFF824
S3150800DB40C4048269DFF8BC04416914F11C05280085
S3150800DB5000F076FADFF8AC048069D0F110010022F3
S3150800DB60DFF8A0048069204410F11C052800FFF79F
S3150800DB703DFE4021002214F12C052800FFF736FE51
S3150800DB808021002214F16C052800FFF72FFE0422DD
S3150800DB90DFF87C14EC34200000F052FA31BD10B5E1
S3150800DBA0DFF8700404682000FFF795FF012114F1DF
S3150800DBB0F000FFF753FFFFF77AFFFFF788FFDFF85C
S3150800DBC054140968411ADFF84C040068FFF7E1FDB0
S3150800DBD010BD10B5DFF83C0404682000FFF77BFF92
S3150800DBE0032114F1F000FFF739FFFFF740FFFFF7B5
S3150800DBF04EFFFFF76CFFDFF81C140968411ADFF8BF
S3150800DC0014040068FFF7C5FD10BDF8B5060006EB5D
S3150800DC100104002509E00422B11CDFF8FC73380072
S3150800DC2000F00EFA70783044861CA64234D230785A
S3150800DC300128F0D003280AD0062810D0332820D08F
S3150800DC40352814D0362814D0FF2822D0EAE7042233
S3150800DC50B11CDFF8C873380000F0F2F9E2E70422D5
S3150800DC60B11CDFF8BC73380000F0EAF9DAE7B578DA
S3150800DC70D8E70422B11CDFF88473380000F0E0F915
S3150800DC80D0E70422B11CDFF89C73380000F0D8F9FD
S3150800DC90C8E72800C0B201E02800C0B2F2BD38B516
S3150800DCA0DFF8700304682078022823D10422DFF8FD
S3150800DCB05813201D01F076F800281BD1DFF844031D
S3150800DCC08269DFF84003416914F11C0001F06AF823
S3150800DCD000280FD1042214F11001DFF8245328007C
S3150800DCE000F0AEF9DFF84003018814F1F000FFF701
S3150800DCF08CFF00E0002032BD10B50120DFF80413C8
S3150800DD000988002916D040F20F12891A25D0491E13
S3150800DD102CD0153960D0491E67D02F3900F0BB804A
S3150800DD20491E00F0C180143900F0DC80491E00F05D
S3150800DD30E28010E10120B34988704FF47A70B14946
S3150800DD400861FFF72CFFAF480169B84801F05BF896
S3150800DD50002040F20F11AB4A1180C0B2002801D151
S3150800DD600320FDE04FF48870A6490880B048007883
S3150800DD70800706D4AD4801F04DF8002801D10020EF
S3150800DD80EEE0AB480078800707D5FFF788FF022842
S3150800DD9003D102209B4988700EE09A4800694EF626
S3150800DDA06021884204DA974800694000954908616D
S3150800DDB0944880780228C4D14FF47A709149086152
S3150800DDC0FFF707FF8F480169984801F01CF8002003
S3150800DDD040F225118B4A1180C0B2002801D10320D8
S3150800DDE0BEE04FF493708749088091480078800711
S3150800DDF006D48E4801F00EF8002801D10020AFE0C5
S3150800DE008B480078800722D5FFF749FF05281ED1E1
S3150800DE1003207C4988707B4800F0DCF87948008C40
S3150800DE20FFF7B0FC04047748408CFFF7ABFC0443CB
S3150800DE3064084FF47A7000FB04F0B0F1004F1CD26E
S3150800DE404FF47A7000FB04F06E49086119E06D48DA
S3150800DE50006942F2117188420ADA6A48006910F5C7
S3150800DE607A7068490861674880780328A8D1D2E79C
S3150800DE70002064490880002072E07FF00040614974
S3150800DE80086160480169694800F0BDFF002040F25A
S3150800DE9055115C4A1180C0B2002801D103205FE009
S3150800DEA04FF4AB7057490880604800F0B3FF00286C
S3150800DEB001D1002054E00220524988704FF47A704C
S3150800DEC05049086100F075F800F0B8F8FFF781FED0
S3150800DED04C480169554800F096FF00204FF4B5718B
S3150800DEE0484A1180C0B2002801D1032038E040F228
S3150800DEF06B10444908804E480078800706D44B4882
S3150800DF0000F088FF002801D1002029E04848007861
S3150800DF1080070AD5FFF7C3FE052806D1032039492D
S3150800DF208870384800F056F878E73648006942F2B3
S3150800DF30117188420ADA3348006910F57A70314956
S3150800DF400861304880780328C0D1EAE700202D49C7
S3150800DF500880002004E0002000202A4908800220CA
S3150800DF6010BD80B5274A50612648816100202549A1
S3150800DF7088704FF6FF70ADF800004FF6FF70ADF8E9
S3150800DF8002004FF486416846FEF73AFA1D49486092
S3150800DF901C484068002804D04FF48840194949684D
S3150800DFA0888000201749088001BD80B5FFF7A4FEC8
S3150800DFB001BD81B00020ADF800000020ADF80200D8
S3150800DFC0BDF8000011490880BDF802000F494880D5
S3150800DFD001B07047818C0D4A1180C18C0B4A518063
S3150800DFE0018D144A1180418D124A5180018E124AC0
S3150800DFF01180408E1049488070470000B487FE1F84
S3150800E000BC87FE1F9887FE1FACFF00083088FE1FDE
S3150800E010B0FF00083C88FE1FC087FE1FC887FE1F8A
S3150800E020C487FE1FB887FE1F5888FE1FA087FE1FDD
S3150800E0306788FE1F3888FE1F3488FE1F7047000059
S3150800E04062B38B0708D0521E11F8013B00F8013B5A
S3150800E05000F024808B07F6D1830740F0208000BFAC
S3150800E060103A07D330B4B1E83810103AA0E838109F
S3150800E070F9D230BC530724BFB1E80810A0E808104D
S3150800E08044BF51F8043B40F8043BD20724BF31F89B
S3150800E090022B20F8022B44BF0B7803707047083A0E
S3150800E0A007D3B1E80810083A40F8043B40F804CB17
S3150800E0B0F7D25307E4E70000CD48016070470168CE
S3150800E0C0096831F4801100680160704703681B68AD
S3150800E0D033F4904309B2194312B211430068016040
S3150800E0E07047416990F8260040010858C00FC0B231
S3150800E0F07047016841F21802895851F00201026816
S3150800E10041F21803D1500168096851F0040100680A
S3150800E11001607047016841F21802895851F40051AC
S3150800E120026841F21803D1500168096851F00801E4
S3150800E1300068016070470221026841F21403D15059
S3150800E1400021006841F2040281507047416990F845
S3150800E15026004001084480687047426990F8260006
S3150800E1604001104441607047E0B55FF4803001908B
S3150800E17000208DF800006A4609219E4800F058FEE6
S3150800E18000208DF800006A4604219B4800F050FEE6
S3150800E19000208DF800006A460221974800F048FEE4
S3150800E1A000208DF800006A460321934800F040FEDF
S3150800E1B000208DF8080088208DF800006A460521A1
S3150800E1C08D4800F035FE00208DF8080088208DF86F
S3150800E1D000006A460821884800F02AFE00208DF8CB
S3150800E1E0080088208DF800006A460921824800F058
S3150800E1F01FFE00208DF800006A4608217D4800F0C1
S3150800E20017FE00208DF8080088208DF800006A4661
S3150800E2100721794800F00CFE00208DF800006A46B8
S3150800E2200021754800F004FE01220021724800F022
S3150800E23087FE5FF080618908890031F00C010220B1
S3150800E24060F30921022060F38B2131F4404101205B
S3150800E25060F397516948FFF72FFF07BD1CB567485C
S3150800E26000F0A3FE6548FFF72AFF00F009F900F55C
S3150800E270985488340021614801F09FF8002803D19A
S3150800E28000F0FEF8A042F5D35D4A00215B4801F094
S3150800E29048F84FF400624FF480415848FFF716FFDC
S3150800E2A05648FFF737FF5548FFF723FF08208DF834
S3150800E2B0000000208DF8010027208DF80200692053
S3150800E2C08DF803005B208DF8040045208DF80500C5
S3150800E2D09DF800004B4908709DF8010049494870AF
S3150800E2E09DF80200474988709DF803004549C870A3
S3150800E2F09DF80400434908719DF805004149487195
S3150800E30013BD082101700021417027218170692100
S3150800E310C1705B21017145214171704738B50024F0
S3150800E320364800F021FF0500002D09D040F2F550CF
S3150800E330854205D22A003449304800F0E0FE2C0018
S3150800E340200032BD80B53148008800284FD02F48BC
S3150800E350008840F2F551884249D22848FFF7C1FEA5
S3150800E360002803D02548FFF7E6FE40E02348FFF7DC
S3150800E370EDFE002103E0244A525C4254491C234A1C
S3150800E38012889142F7D3214801881C48FFF7E5FE19
S3150800E3901A4890F82600194981F828001748406954
S3150800E3A0164991F826104901144A5269134B93F8F5
S3150800E3B026305B01D25852F0004242500F4890F87E
S3150800E3C02600401C0D4981F826000C4890F82600C6
S3150800E3D00A4991F82510884203D10020074981F897
S3150800E3E026000020054908620448FFF7A4FE01BD7F
S3150800E3F040400050008F0248008202484080FE1FBD
S3150800E4009CFF00081888FE1F7080FE1F5888FE1F94
S3150800E41040B2002808D589001E4A40B210F00F0005
S3150800E420104400F8041C03E089001B4A40B211544A
S3150800E430704780B5411EB1F1807F01D301200EE0FF
S3150800E440401E164908603F215FF0FF30FFF7E0FFE6
S3150800E450002013490860072012490860002002BD01
S3150800E46080B5114800684FF47A71B0FBF1F0FFF7F8
S3150800E470E0FF002000F001F801BD0C490860704774
S3150800E4800A480068704709480068401C0749086040
S3150800E4907047000018ED00E000E400E014E000E03A
S3150800E4A018E000E010E000E08088FE1F2C88FE1FC0
S3150800E4B080B500F024F800280DD1334833490860A8
S3150800E4C0002004E00021314A02441171401C38281A
S3150800E4D0F8D300F023F801BD70B504000D0000263E
S3150800E4E000F00DF8002807D0382C05D2274820441C
S3150800E4F0057100F013F801263000C0B270BD10B5E2
S3150800E5000024224800682049884204D100F00CF80B
S3150800E510002800D001242000C0B210BD80B500F04C
S3150800E52010F81A49888701BD10B5002400F009F8CB
S3150800E5301649898F80B2884200D101242000C0B2D2
S3150800E54010BD00201149096850FA81F00F49096881
S3150800E550090A50FA81F00D490968090C50FA81F048
S3150800E5600A490968090E50FA81F0002105E0074AB0
S3150800E5700A44127950FA82F0491C3829F7D380B236
S3150800E580C043401C80B27047A2E742CE0080FE1FFF
S3150800E590BFF34F8FDFF88803006810F4E060DFF8F8
S3150800E5A084130843DFF878130860BFF34F8F00BF62
S3150800E5B0FDE7C9B200EB8103DB69DB08DB00D2B2F9
S3150800E5C01A43C9B200EB8100C2617047D0F8140142
S3150800E5D0C00810F001007047016C0909090151F0E3
S3150800E5E0020101647047C268D208D200C9B211F0AC
S3150800E5F007011143C1607047016851F0400101608D
S3150800E6007047016831F0400101607047016851F0B8
S3150800E61001010160704701684908490001607047B7
S3150800E6200068C06970470068C1617047816851F029
S3150800E630005181600168C96851F000510068C160E5
S3150800E640704780B500F00DF800F0ACF801BD80B554
S3150800E65000F04FF800F034F901BD80B5FFF798FFD8
S3150800E66001BD00B589B04FF46140009008208DF8CF
S3150800E670040008208DF8050001208DF806001020FA
S3150800E6808DF807000020ADF808006946A64800F096
S3150800E690A1FE00208DF818000120079002208DF8B1
S3150800E6A0200006AA0421A14800F0C2FB90208DF89C
S3150800E6B00C000120049002208DF8140003AA0521FD
S3150800E6C09A4800F0B5FB012200219748FFF771FF31
S3150800E6D0012304221021944800F02BFF0123042271
S3150800E6E00021914800F03AFF8F48FFF775FF09B0FF
S3150800E6F000BD80B58E480078002817D18D4800F0F7
S3150800E70042F801283ED18B48007800283AD089483B
S3150800E7100078412836DAFFF7B3FE874908600120FA
S3150800E720834908700020854908702BE08148834991
S3150800E73009780844401C00F026F8012818D17F48BB
S3150800E7400078401C7D4908707C480078794909782A
S3150800E750884217D100207649087076484078FF2805
S3150800E76010D17448807800280CD1FFF776FF09E0AD
S3150800E770FFF786FE704909686431814202D200209B
S3150800E7806B49087001BD10B504006748FFF71EFF06
S3150800E790002805D1644800F05AFE2070012000E0E8
S3150800E7A0002010BD10B58AB000F039FF040000E063
S3150800E7B0640063488442FBD36248844201D36408F8
S3150800E7C0FAE722000121604801F03CF800945F480E
S3150800E7D001904FF4FA50ADF808000120ADF80A0090
S3150800E7E069465B4800F064FF5948FFF705FF58483B
S3150800E7F0FFF70CFF574858490860022056494968F0
S3150800E80060F39F715448416040F2676020F0004011
S3150800E8105149496860F31C014F4A51604E4989685D
S3150800E82060F31C014C4881604B48406830F000504A
S3150800E830494948604848FFF7F9FE082046490873E1
S3150800E840002005E00021444AC0B202441174401C6D
S3150800E8500100414A127BC9B29142F3D300203E49D6
S3150800E86008763D4801F04BF801220121364800F0B0
S3150800E870B5FF3748FFF7C5FE3548FFF7CCFE002041
S3150800E8808DF8180006AA0D21284800F0D1FA902024
S3150800E8908DF80C000120049002208DF8140003AABC
S3150800E8A00C21224800F0C4FA2948FFF7A5FE0221E8
S3150800E8B02748FFF798FE2648FFF7A3FE0AB010BDC3
S3150800E8C01CB500242448FFF7ABFEC00719D522481B
S3150800E8D001F090F8002810D1002008E01E49C0B2C7
S3150800E8E00144097C6A46C0B211540124401C010047
S3150800E8F0194A127BC9B29142F0D301211648FFF793
S3150800E90092FEE4B2012C0AD100249DF80000FF28EB
S3150800E91005D19DF80100002801D1FFF79EFE13BD21
S3150800E9200CED00E00400FA050000034000810248EF
S3150800E9306588FE1F1487FE1FCC87FE1F6488FE1F8E
S3150800E940001BB700010E27070040014820A1070059
S3150800E9500043014820500148D087FE1F10B5DFF854
S3150800E960FC030078401CDFF8F41308700020DFF879
S3150800E970E413087020E0DFF8E003DFF8D81309781D
S3150800E9800C22514300EB01042088618808430028C3
S3150800E9900BD0DFF8C8030078A17A401A782804DB80
S3150800E9A0042100222000FEF721FFDFF8A8030078E3
S3150800E9B0401CDFF8A0130870DFF8980300780828D1
S3150800E9C0D9DB10BD70B50C00DFF88C530021DFF8D9
S3150800E9D08423117006E0DFF87C130978491CDFF8F8
S3150800E9E074231170DFF86C130978082921DADFF827
S3150800E9F06813DFF8602312780C235A4301EB0205EB
S3150800EA0029880029E7D069880029E4D001882A885E
S3150800EA109142E0D141886A889142DCD106222E1DB6
S3150800EA2021003000FFF70CFBDFF830030078A872EE
S3150800EA306BE00021DFF81C23117006E0DFF81413E1
S3150800EA400978491CDFF80C231170DFF808130978D8
S3150800EA5008290EDADFF80013DFF8F82212780C23FB
S3150800EA605A4301EB020529880029E7D1698800295C
S3150800EA70E4D1DFF8E0120978082938D10021DFF857
S3150800EA80E02211700021DFF8DC2211700021B14A62
S3150800EA9011701DE0B049AF4A12780C235A4301EBB6
S3150800EAA00205AF490978AD4A1278AB7AD21A914273
S3150800EAB009DAAA490978AA7A891AA94A1170A549C8
S3150800EAC00978A84A1170A3490978491CA14A117006
S3150800EAD0A04909780829DDDBA24909789D4A117001
S3150800EAE09D499C4A12780C235A4301EB02050422DD
S3150800EAF001002800FFF7A4FA06222E1D2100300087
S3150800EB00FFF79EFA95480078A87270BD10B596482A
S3150800EB1000882A2803D20020934908805FE0002055
S3150800EB20914908809148808AB0F5807F03D0B0F576
S3150800EB30007F44D053E08D48C08C8D4909888842AF
S3150800EB403CD18A48008D8A494988884236D1894904
S3150800EB508948FFF737FF4FF40070844988820622F8
S3150800EB608449864C2000FFF76BFA06228449814CBB
S3150800EB702000FFF765FA06228149824C2000FFF73C
S3150800EB805FFA06227D49794C2000FFF759FA774843
S3150800EB90808B7649C8847548C08B74490885744843
S3150800EBA0008872498883724840887049C8834FF440
S3150800EBB0C1606E4988812A206B4908800FE06B483E
S3150800EBC0C08C6B490988884209D16848008D684914
S3150800EBD04988884203D167496748FFF7F3FE10BDA5
S3150800EBE010B55D486149C98B674A128891420CD1B4
S3150800EBF05E49098C644A5288914206D106226349C5
S3150800EC005A4C2000FFF71CFA93E05849C98B604A12
S3150800EC1012881140564A12885D4B1B881A40914249
S3150800EC200BD15249098C5A4A52881140504A528887
S3150800EC30574B5B881A40914208D056490988564A6C
S3150800EC40118054494988544A518007E04749C98B7D
S3150800EC50514A11804549098C4F4A518000213D4A45
S3150800EC60117004E03B490978491C3A4A1170394940
S3150800EC70097808290FDA3848364909780C225143A9
S3150800EC8008444549098802889142EBD14249498896
S3150800EC9042889142E6D12F490978082943D10621AD
S3150800ECA0FF22324C2000FEF7A1FD06210022334C3C
S3150800ECB02000FEF79BFD06223149324C2000FFF763
S3150800ECC0BFF906222E492B4C2000FFF7B9F9324826
S3150800ECD000882649C884304840882449088524483D
S3150800ECE0008822498883224840882049C8834FF4EF
S3150800ECF080701E4988824FF480701C49C88108209C
S3150800ED001A49088206201949887404201749C874C4
S3150800ED104FF4C160154988812048214908602A2096
S3150800ED201149088013E00622011D104C2000FFF748
S3150800ED3087F906221249134C2000FFF781F90820AB
S3150800ED400A498881084800880E300749088010BD9E
S3150800ED50000000006A88FE1FB486FE1F6C88FE1F2E
S3150800ED606D88FE1F6B88FE1F5888FE1F7080FE1F69
S3150800ED703088FE1F8680FE1F8C80FE1F9080FE1F37
S3150800ED801888FE1F7680FE1FBCFF0008A4FF000837
S3150800ED903888FE1F3488FE1F5488FE1FA680FE1F73
S3150800EDA03C88FE1F0300002013F0030F09D0521EF3
S3150800EDB022BF13F8010B11F801CBB0EB0C00F3D00E
S3150800EDC07047121F22BF53F8040B51F804CB604555
S3150800EDD0F7D0121D0AD200BA9CFA8CFCB0EB0C00D4
S3150800EDE038BF6FF0000088BF01207047521E22BF4F
S3150800EDF013F8010B11F801CBB0EB0C00F6D0521C3E
S3150800EE0008BF1046704710B50400616000F028FE80
S3150800EE10206010BD10B5040000F022FE2168401ADB
S3150800EE206168884201DB012000E00020C0B210BD05
S3150800EE3070B4C9B28B1000EB8303C9B28C1000EB17
S3150800EE4084042469F82511F00306F6B2F600B540E5
S3150800EE50AC431C61436F03244D00AC40A343436796
S3150800EE60224B984202D0224B984205D1036E0124C8
S3150800EE708C40A343036624E053688B404360C9B2C1
S3150800EE80CB1000EB8303C9B2CC1000EB8404246CCE
S3150800EE90072511F00706F6B2B600B540AC431C6468
S3150800EEA0C9B2CB1000EB8303C9B2CC1000EB8404C3
S3150800EEB0246C157A11F00706F6B2B600B5402C4355
S3150800EEC01C64C9B28B1000EB8303C9B28C1000EB2B
S3150800EED084000069127811F00301C9B2C90012FA58
S3150800EEE001F10843186170BC70470000008E0248A3
S3150800EEF0008F024870B4C9B28B0800EB8303C9B20D
S3150800EF008C0800EB84042469F82511F00306F6B290
S3150800EF10F600B540AC431C61C9B28B0800EB83030D
S3150800EF20C9B28C0800EB84000069D2B211F0030163
S3150800EF30C9B2C90012FA01F10843186170BC7047DA
S3150800EF4030B4436F03244D00AC40A3434367436F7B
S3150800EF50D2B2490012FA01F11943416730BC704731
S3150800EF6001684FF48052895851F0010102684FF444
S3150800EF708053D15001684FF480528958C907F9D493
S3150800EF80704701680B64006842647047DFF8100335
S3150800EF900068DFF81013096811F00101884070470E
S3150800EFA080B5FFF7F3FF400802BD38B5040020001E
S3150800EFB000F026F92000FFF7D3FF200000F0EBF859
S3150800EFC00500D4E902232000FFF7DBFF4FF4806039
S3150800EFD021680860802021688861DFF8CC022168F2
S3150800EFE041F218028850DFF8C40221684FF48052B3
S3150800EFF08850200000F021F8200000F052F85FF059
S3150800F000FF30216841F2140288507FF07C40216865
S3150800F010C1F810017FF07C402168C1F80C017FF02F
S3150800F020C0202168C1F800024FF402702168C86345
S3150800F030002020622800C0B232BD10B4002122E0B0
S3150800F0405FF0004203694C011A5102694B011A44E8
S3150800F05044F2F453536002694B011A44836940F23F
S3150800F060F45404FB01F4234493604A1C90F82430BA
S3150800F0709A4200D1002203694C01234404695201D3
S3150800F0802244DA60491C90F824209142D8D30169B9
S3150800F090026841F20C03D150002180F8271010BCF9
S3150800F0A0704710B400211CE0DFF8042243694C01C4
S3150800F0B01A5142694B011A44C36940F2F45404FBDD
S3150800F0C001F4234493604A1C90F825309A4200D1F3
S3150800F0D0002243694C012344446952012244DA6000
S3150800F0E0491C90F825209142DED34169026841F215
S3150800F0F01003D150002180F8261010BC704770B557
S3150800F10004000E001500206994F8271049010844E8
S3150800F11081682A003000FEF793FF206994F82710CB
S3150800F12049015FF00042425094F82700401C84F8D9
S3150800F130270094F8270094F82410884202D100206A
S3150800F14084F82700206841F214014058000609D5C2
S3150800F1508020216841F2140288500020216841F27B
S3150800F16008028850280070BD0021016990F8270020
S3150800F17040010858002801D500210AE010F403418F
S3150800F180B1F5407F02D05FF0FF3102E0C0F30D40D9
S3150800F190011F0800704710B50400FFF701FF0100C2
S3150800F1A0002022681032DFF80C31994202D2082179
S3150800F1B0116023E0DFF80031994202D20C21116078
S3150800F1C01CE0DFF8F830994202D20021116015E000
S3150800F1D0DFF8EC30994202D2042111600EE0DFF824
S3150800F1E0E430994202D21021116007E0DFF8D830E6
S3150800F1F0994202D21421116000E00220C0B210BD6B
S3150800F20080B5042000F015FADFF8C00000F016FA01
S3150800F210DFF8B80000F0FAF901BD10B404682469F3
S3150800F22014F03C04C9B254EAC121D2B251EA82119F
S3150800F23051F0010102681161002102681269D207C2
S3150800F24004D4006840691880002005E0491C4FF680
S3150800F250FF729142F1D3022010BC704710B49BB2E2
S3150800F2600468636103681B6913F03C03C9B253EA77
S3150800F270C121D2B251EA821151F00301026811612B
S3150800F280002102681269D20701D4002005E0491C52
S3150800F2904FF6FF729142F4D3022010BC704700006B
S3150800F2A08088FE1F104600500400200280200102BC
S3150800F2B000001030C10E16020187930301E1F5051F
S3150800F2C081D1F00801C2EB0B81B2E60E04000020E2
S3150800F2D038B504000D000DF1020302222900C9B257
S3150800F2E02000FFF79AFF002818D16B460322290051
S3150800F2F0C9B22000FFF791FF00280FD1BDF8020020
S3150800F300222809D1BDF800004FF6F0710840B0F583
S3150800F310AB5F01D1002002E0032000E00420C0B268
S3150800F32032BD70B504000D0016002900C9B22000D0
S3150800F330FFF7CEFF002826D12900C9B2200000F029
S3150800F34023F800281FD10023B6F90200B0F5804F34
S3150800F35001D153F40053B6F90400B0F5006F01D19A
S3150800F36053F48073B079002801D053F48053F079B0
S3150800F370002801D053F480439BB200222900C9B269
S3150800F3802000FFF76BFF70BD38B504000D004FF481
S3150800F390004300222900C9B22000FFF75FFF0028BA
S3150800F3A00AD16B4600222900C9B22000FFF735FFB3
S3150800F3B0BDF800100904F4D432BD80B56B460122AD
S3150800F3C0C9B2FFF72AFFBDF80000C0B2800810F0E6
S3150800F3D0010002BD70B504000D001026200000F0E3
S3150800F3E041F8E879002800D0EE7932002968200033
S3150800F3F000F061F8A879401EB11CC901090A090282
S3150800F40051EA400040F4403050F00100E0632879AA
S3150800F410401E000650F4817060636879002806D0A3
S3150800F420606B6979491E50EA0140606305E0606BCC
S3150800F4302979491E50EA014060634FF4A060A06331
S3150800F4405FF0FF30E064B5F90800206470BDD0F8BD
S3150800F4500C1111F0E06F01D1406D01E0D0F81C01EC
S3150800F46080B2704710B504005848844202D0584804
S3150800F470844203D1574800F088F812E0564884427F
S3150800F48002D05648844203D1554800F07EF808E079
S3150800F4905448844202D05448844202D1534800F06A
S3150800F4A074F80320E060E068C007FCD5206C00090A
S3150800F4B00001206410BDF8B504000E001500642E86
S3150800F4C034D3002D32D000F0AAF86421B0FBF1F154
S3150800F4D06420B6FBF0F60123012040F2FF3E40F21D
S3150800F4E0FF3212E002FB01F705FB06FCB7FBFCF74F
S3150800F4F05FEA972CBF05BF0DBCF5806F04D2774530
S3150800F50002D2BE4660461300521E002AEAD153F4C0
S3150800F510004121616169364A11406A1E51EA822119
S3150800F520401E51EA00406061002000E00120C0B2A0
S3150800F530F2BD30B4D0F8084134F0E064C0F80841B0
S3150800F540D0F808412B4D2C4054EA03231943D2B274
S3150800F55051EA0261C0F8081130BC704730B4D0F8DF
S3150800F5600C4134F0E064C0F80C41D0F80C41224D4F
S3150800F5702C4054EA03231943D2B251EA026151F0EE
S3150800F5808051C0F80C1130BC704780B511498842CB
S3150800F59008D14FF4006000F051F84FF4006000F015
S3150800F5A035F812E00E49884206D1144800F046F8AC
S3150800F5B0124800F02BF808E00C49884205D110489B
S3150800F5C000F03CF80E4800F021F801BD00000340A9
S3150800F5D000020340080003400000024800020248F7
S3150800F5E00800024800400248004202480840024813
S3150800F5F0EF8000FCC0C0FFF8C0C0FFEF800000101D
S3150800F60000010010DFF8480000687047010F20F07D
S3150800F6107040DFF840200C2359435050704780B59E
S3150800F620FFF7F0FFDFF83010096811F00101C84054
S3150800F63002BDC0B2DFF8241008607047010F20F041
S3150800F6407040DFF81C200C235943505070470000C7
S3150800F6508088FE1F1444005014460050044600508B
S3150800F66048460050D0F8C40110F4407F01D101206B
S3150800F67000E00020C0B27047C9B2D2B251EA0241D6
S3150800F680DBB251EA0361C0F8C4117047016851F052
S3150800F690400101607047016831F040010160704720
S3150800F6A0814200D308007047884200D3080070479B
S3150800F6B02DE9F04104000D000C220C22002601273A
S3150800F6C05FF00008002042F21071012200E0521C8F
S3150800F6D0412A40D22B685FF00A0C0CFB03F3B3FBFC
S3150800F6E0F2FC6B68BCFBF3F35FF00A0EB3FBFEF8A3
S3150800F6F00EFB183EBEF1060F05D35FF00A0EB3FBEC
S3150800F700FEF35B1C03E05FF00A0EB3FBFEF3002B6F
S3150800F71006D05FF00A0E0EFB03FEBCFBFEFC03E000
S3150800F7200A23BCFBF3FC0123D5F804E0F44504D313
S3150800F730D5F804E0BCEB0E0C03E0D5F804E0BEEB0C
S3150800F7400C0C152BC3D28C45C1D216001800614685
S3150800F750BCF57A7FBBD242F21071402200E0521EFD
S3150800F760032A1BD3531C42F2107C0CFB03F3B3FB96
S3150800F770F0F3B5F808C0634504D3B5F808C0B3EB91
S3150800F7800C0C03E0B5F808C0BCEB030C8C4501D2A1
S3150800F79017006146B5F808C06345E0D2C01BB0F152
S3150800F7A001082000FFF772FFB8F10100000310F40A
S3150800F7B0E0406989491E890111F0C0010843791E94
S3150800F7C0090211F470610843711E11F03F010843E4
S3150800F7D020612000FFF75FFFBDE8F08170B50400E7
S3150800F7E00D0016002000FFF73DFF0028FAD06B1C1D
S3150800F7F0DBB23200D2B202212000FFF73DFF70BD16
S3150800F80010B50400DFF84402FFF718FFDFF83C02E2
S3150800F810FFF7FCFE2068400840002060206880074B
S3150800F820FCD410BD80B500F065F8012802D0022886
S3150800F83003D005E0FFF7F3FE03E000F015F900E05A
S3150800F840002002BD2DE9F04104000E00150020003D
S3150800F850FFF7D6FF3100C9B2200000F042F82000B9
S3150800F860FFF7E0FF8046B8FBF5F0D0F58061002091
S3150800F870FFF716FF40F2FF31FFF716FF0600D6F531
S3150800F8808060B8FBF0F7A8095FEA981840F2FF31E4
S3150800F8904FF480625043B0FBF8F0FFF705FF00FB1A
S3150800F8A008F1890A8901691AEA1B914201D30121E3
S3150800F8B000E00021C9B2002900D10600C9B200291A
S3150800F8C001D0012000E00220E168DFF88421114020
S3150800F8D0E160E168C0B256EA80300843E060BDE8FE
S3150800F8E0F081D0F8C82112091201C9B21143C0F833
S3150800F8F0C8117047D0F8C80110F00F00704710B54E
S3150800F90004002068DFF84C11081840094109000274
S3150800F91010F4F85050EA41302168896831F47F4183
S3150800F9202268916021688968084321688860606850
S3150800F930C0F34070C00704D56068C0F34070C007C4
S3150800F94036D5207E002802D0207E012830D12020FE
S3150800F9502168C8616068C0F34070002810D16068EB
S3150800F96010F06040616850EA814021688861A068AB
S3150800F97010F06040A16850EA81402168C86005E03F
S3150800F980606821688861A0682168C860207E0128AF
S3150800F99007D1200000F00DF85FF000602168C8610B
S3150800F9A003E04FF400602168C8612B482168C861EC
S3150800F9B010BD0321017E012918D120210268D161D9
S3150800F9C00168096831F07061027B120612F07062F4
S3150800F9D01143026811600169026811614169026890
S3150800F9E051611E490068C161002100E00321080039
S3150800F9F0C0B270470121002100220168C969C1F31C
S3150800FA00C0210268D269C2F38002002901D003210D
S3150800FA1018E0012A01D1022114E00168096901618F
S3150800FA200168496941610168C969C1F380010268D1
S3150800FA30D269C2F3C002C9B2002902D0D2B2002AE2
S3150800FA40EBD100210800C0B270470000100000107A
S3150800FA50003CFFFF00B0FEB74000A00640002800AB
S3150800FA6080B5FEF70DFD02BD00487047001BB700C4
S3150800FA7080B566480068C00709D46548006850F034
S3150800FA8001006349086061480068C007FBD5614802
S3150800FA900068800509D56048006850F400705E4922
S3150800FAA0086041F64C5000F0EBF85C48006850F4EA
S3150800FAB000205A49086040F6C41000F0E1F857489B
S3150800FAC0006857490840554908605648006810F0CC
S3150800FAD0300F24D0534800685349084051490860FC
S3150800FAE0FFF7C2FF4F490968504AB0FBF2F0401EC3
S3150800FAF051EA00404B4908604D48006840084000FC
S3150800FB004B4908604548006830F4003043490860AE
S3150800FB104848006810F46070B0F5607FF8D13F4837
S3150800FB20006850F001003D4908603C48006850F004
S3150800FB3010003A490860404840490860374800685C
S3150800FB4050F04000354908603448006830F010002D
S3150800FB50324908603148006850F480202F4908600F
S3150800FB60344800684007FBD52C4800684008400028
S3150800FB702A4908602F480068C007FBD45FF00110C7
S3150800FB802F49086000202F49086000202E49086088
S3150800FB9000202E49086000202D49086003202D49C1
S3150800FBA008602D482D4908602D482E4908601B48D5
S3150800FBB0006830F04000194908602B481F49086062
S3150800FBC04FF4166000F05CF828481C4908604FF4AA
S3150800FBD0616000F055F82648184908604FF49650B9
S3150800FBE000F04EF823481549086041F2707000F09D
S3150800FBF047F82148114908604FF4E15000F040F8F1
S3150800FC0000201E49086000F059F801BD0042005066
S3150800FC100442005000440050084400501447005065
S3150800FC20FDFFFEFF04470050CFFFF0FFA02526008A
S3150800FC301C47005010470050002F0B011847005072
S3150800FC400C460050144600501046005020460050FE
S3150800FC50244600501C460050050001001846005076
S3150800FC600300200128460050002F0501002F03013C
S3150800FC70002F0201002F0101002F00010446005049
S3150800FC8081B00021009103E000BF0099491C009152
S3150800FC9000998142F8D301B07047000010B51022D0
S3150800FCA05FF00051044C2000FEF7CAF900F054F842
S3150800FCB0FFF7DEFE10BD00BF7088FE1F80B51F4827
S3150800FCC00068C00327D51E480068C00701D51D482F
S3150800FCD001E0FFF7C9FE1C490968490713D51B4906
S3150800FCE00968C1F30361491C184A1268C2F306225F
S3150800FCF0521C164B1B68C3F306435B1C5943B0FBE7
S3150800FD00F1F0504308E01149096811F07F014B1CD6
S3150800FD10B0FBF3F000E00B480849096801F0FF0161
S3150800FD20491CB0FBF1F00A49096811F00101491CA8
S3150800FD30B0FBF1F00749086001BD00BF0C46005052
S3150800FD401C47005000366E011047005018470050F7
S3150800FD50104600508088FE1F72B60D480D4908608F
S3150800FD60BFF34F8F62B60C48006850F470000A491A
S3150800FD7008600A48006830F0080008490860084822
S3150800FD8000680009000150F0040005490860704742
S3150800FD9000C0000808ED00E088ED00E014ED00E082
S3150800FDA01420005812FA01F14160704780B580228C
S3150800FDB008211648FFF79EF85FF480320821134899
S3150800FDC0FFF7F0FF01BD10B5FEF75AFB0400104817
S3150800FDD00068201AB0F5FA7F17D30E480078002875
S3150800FDE008D101200B490870012208210748FFF7AE
S3150800FDF0D9FF08E00020074908705FF4803208211F
S3150800FE000248FFF7CFFF0248046010BD008502488C
S3150800FE102088FE1F6688FE1F19E050F8041BCB07D2
S3150800FE2044BFA9F101035918121F0023042A41F8F7
S3150800FE30043BF9D25FEA827C0B4604D54FF0000CEE
S3150800FE40A1F800C09B1CD10744BF0021197050F8C7
S3150800FE50042B002AE1D1704780B500F011F8FEF7AF
S3150800FE6027FBFDF7F7FCFEF7ECFB00210020FEF769
S3150800FE7033FBFFF7A8FFFDF752FDFEF7E8FBF8E7AF
S3150800FE8080B5FFF71BFFFFF791FFFEF7E9FA01BD03
S3150800FE9010B450F8041B79B102684368024408306C
S3150800FEA0DC0744BFA9F10104E31852F8044B43F8F0
S3150800FEB0044B091FF9D1ECE710BC704710B5074988
S3150800FEC079441831064C7C44163404E00A68081D47
S3150800FED0114488470146A142F8D110BD2C00000004
S3150800FEE0540000004EF68851CEF20001086840F42E
S3150800FEF070000860BFF34F8FBFF36F8F4FF000702D
S3150800FF00E1EE100A7047000011FFFFFF000800002D
S3150800FF107080FE1FA03000000000002000000000D6
S3150800FF2071FFFFFF300000004C0200004080FE1FFA
S3150800FF300000000000F00BF8002801D0FFF7BEFF14
S3150800FF400020AFF30080FFF787FF00F002F80120DA
S3150800FF50704700F001B800000746384600F002F87E
S3150800FF60FBE7000080B5AFF30080024A11001820B5
S3150800FF70ABBEFBE726000200DFF808D00248804740
S3150800FF80024800478890FE1F9DFC000891FF000864
S3150800FF90AFF30080FFF7A6FFFFF7CCFF0100004094
S3150800FFA000080000FFFFFFFFFFFF0000ADDE122381
S3150800FFB063825363FFFFFFFF00000000FFFFFFFFA0
S3150800FFC0FFF7FEBFFFF7FEBFFFF7FEBFFFF7FEBF57
S3150800FFD0FFF7FEBFFFF7FEBFFFF7FEBFFFF7FEBF47
S3150800FFE0FFF7FEBFFFF7FEBFFFF7FEBFFFF7FEBF37
S3150800FFF0FFF7FEBFFFF7FEBFFFF7FEBFFFF7FEBF27
S31508010000FFF7FEBFFFF7FEBFFFF7FEBFFFF7FEBF15
S31508010010FFF7FEBFFFF7FEBFFFF7FEBFFFF7FEBF05
S31508010020FFF7FEBFFFF7FEBFFFF7FEBFFFF7FEBFF5
S31508010030FFF7FEBFFFF7FEBFFFF7FEBFFFF7FEBFE5
S31508010040FFF7FEBFFFF7FEBFFFF7FEBFFFF7FEBFD5
S31508010050FFF7FEBFFFF7FEBFFFF7FEBFFFF7FEBFC5
S31508010060FFF7FEBFFFF7FEBFFFF7FEBFFFF7FEBFB5
S31508010070FFF7FEBFFFF7FEBFFFF7FEBFFFF7FEBFA5
S31508010080FFF7FEBFFFF7FEBFFFF7FEBFFFF7FEBF95
S31508010090FFF7FEBFFFF7FEBFFFF7FEBFFFF7FEBF85
S315080100A0FFF7FEBFFFF7FEBFFFF7FEBFFFF7FEBF75
S315080100B0FFF7FEBFFFF7FEBFFFF7FEBFFFF7FEBF65
S315080100C0FFF7FEBFFFF7FEBFFFF7FEBFFFF7FEBF55
S315080100D0FFF7FEBFFFF7FEBFFFF7FEBFFFF7FEBF45
S315080100E0FFF7FEBFFFF7FEBFFFF7FEBFFFF7FEBF35
S315080100F0FFF7FEBFFFF7FEBFFFF7FEBFFFF7FEBF25
S31508010100FFF7FEBFFFF7FEBFFFF7FEBFFFF7FEBF14
S31508010110FFF7FEBFFFF7FEBFFFF7FEBFFFF7FEBF04
S31508010120FFF7FEBFFFF7FEBFFFF7FEBFFFF7FEBFF4
S31508010130FFF7FEBFFFF7FEBFFFF7FEBFFFF7FEBFE4
S31508010140FFF7FEBFFFF7FEBFFFF7FEBFFFF7FEBFD4
S31508010150FFF7FEBFFFF7FEBFFFF7FEBFFFF7FEBFC4
S31508010160FFF7FEBFFFF7FEBFFFF7FEBFFFF7FEBFB4
S31508010170FFF7FEBF00C00050000000000800276915
S315080101805B450000A02F0020203000200000002041
S31508010190D017002000000000040400000000000041
S309080101A0000000004C
S7050800FF9162
